:020000000428D2
:08000800FF30A200FF30A3004D
:10001000FF30A400FF30A5000F30A6008A110A129D
:100020007A270A308A110A129B2727128A110A128C
:10003000FC2703308A110A12692732308A110A120A
:10004000C72703308A110A12692732308A110A122F
:10005000C72703308A110A12692732308A110A121F
:10006000C72732308A110A12532728308A110A1200
:1000700053278A110A120D278A110A12BD268A11E6
:100080000A12092724138A150A121E20A4178A159A
:100090000A121B208A150A124320243098001930B6
:1000A00099008A150A124620903098001A081A08FA
:1000B0001A0800309900AA01AB01A4128A150A128D
:1000C000212023138A150A122D20A3138A150A1240
:1000D0002A20A8168A110A12EA2701308A110A1268
:1000E0009227A8128A110A12EA278A110A12C12439
:1000F000FF308A150A1236208A110A120719A32A1C
:1001000001308A110A1292278A110A120719A32AAA
:10011000A8168A110A12EA2701308A110A129227B8
:10012000A8128A110A12EA278A110A1225278A11AF
:100130000A1207199E288A110A12972801308A117B
:100140000A129227B301B2018A110A120719AB28C9
:100150008A110A127C2A1F3033028A110A12031CE8
:10016000B828A7178A110A12F3278A110A12BC2885
:10017000A7138A110A12F327B101FF308A110A125C
:10018000D025FF30B10700308A110A128F258A115D
:100190000A12212741308A110A1245272A08B7007E
:1001A0002B088A110A128B243408AE003508AF00E0
:1001B0003608B0002F088A110A12D0252F08B1077F
:1001C00030088A110A12D0253008B1071F303302D7
:1001D0008A110A1203180E29AE30B4003308B50094
:1001E0003208B6002F088A110A12DB2501308A1165
:1001F0000A129B278A110A125524AE30B400330824
:10020000B5003208B60030088A110A12DB25013029
:100210008A110A129B278A110A1255242F08B4004A
:1002200030088A110A12622401308A110A128F25BD
:1002300042308A110A1245272A08B7002B088A1172
:100240000A128B243408AE003508AF003608B0001F
:100250002F088A110A12D0252F08B10730088A11F9
:100260000A12D0253008B1071F3033028A110A1252
:1002700003185C29AE30B4003308B5003208B6006C
:100280002F088A110A12DB2501308A110A129B27D6
:100290008A110A125524AE30B4003308B500320872
:1002A000B60030088A110A12DB2501308A110A12C1
:1002B0009B278A110A1255242F08B40030088A118E
:1002C0000A12622402308A110A128F2543308A11E1
:1002D0000A1245272A08B7002B088A110A128B2414
:1002E0003408AE003508AF003608B0002F088A1178
:1002F0000A12D0252F08B10730088A110A12D0251A
:100300003008B1071F3033028A110A120318AA29D4
:10031000AE30B4003308B5003208B6002F088A1199
:100320000A12DB2501308A110A129B278A110A1250
:100330005524AE30B4003308B5003208B60030089A
:100340008A110A12DB2501308A110A129B278A11B1
:100350000A1255242F08B40030088A110A126224A8
:100360008A110A121D2703308A110A128F25443080
:100370008A110A1245272A08B7002B088A110A1287
:100380008B243408AE003508AF003608B0002F08C3
:100390008A110A12D0252F08B10730088A110A12D3
:1003A000D0253008B1071F3033028A110A12031812
:1003B000FB29AE30B4003308B5003208B6002F0870
:1003C0008A110A12DB2501308A110A129B278A1131
:1003D0000A125524AE30B4003308B5003208B60016
:1003E00030088A110A12DB2501308A110A129B2774
:1003F0008A110A1255242F08B40030088A110A12F3
:10040000622404308A110A128F2545308A110A129B
:1004100045272A08B7002B088A110A128B243408B2
:10042000AE003508AF003608B0002F088A110A1256
:10043000D0252F08B10730088A110A12D0253008BC
:10044000B1071F3033028A110A120318492AAE304D
:10045000B4003308B5003208B6002F088A110A121A
:10046000DB2501308A110A129B278A110A125524B2
:10047000AE30B4003308B5003208B60030088A1137
:100480000A12DB2501308A110A129B278A110A12EF
:1004900055242F08B40030088A110A126224203033
:1004A0008A110A12452752308A110A12452745300F
:1004B0008A110A12452743308A110A12452731084A
:1004C000F039AD002D088A110A12D02531080F39F4
:1004D000AD002D088A110A12D02527178A110A1299
:1004E000F62701308A110A12922727138A110A125D
:1004F000F6278A110A12A428A8168A110A12EA27D6
:1005000001308A110A129227A8128A110A12EA27C8
:10051000AE30B4003308B5003208B600FF308A119F
:100520000A12DB2501308A110A129B278A110A124E
:1005300025278A110A12C1248A110A120719A32A2F
:100540008A110A129C2A8A110A1287184F2C01302C
:100550008A110A1292278A110A1287184F2CA8169C
:100560008A110A12EA2701308A110A129227A81268
:100570008A110A12EA278A110A1225278A110A12F9
:100580008718C52A8A110A12BE2A01308A110A1256
:1005900092278A110A12252727178A110A12F6278D
:1005A000B301B2011F3033028A110A120318DC2A88
:1005B0008A110A128718DF2A8A110A12322CB10115
:1005C000FF308A110A12D025FF30B107AE30B400D7
:1005D0003308B5003208B6008A110A12F825370828
:1005E000A9002908AF008A110A125524AE30B400C0
:1005F0003308B5003208B6008A110A12F825370808
:10060000A9002908B0008A110A1255248A110A1279
:10061000212741308A110A1245272F088A110A1210
:10062000D0252F08B10730088A110A12D0253008CA
:10063000B1072F08B40030088A110A126224AE30C4
:10064000B4003308B5003208B6008A110A12F82542
:100650003708A9002908AF008A110A125524AE30C4
:10066000B4003308B5003208B6008A110A12F82522
:100670003708A9002908B0008A110A12552442300F
:100680008A110A1245272F088A110A12D0252F082D
:10069000B10730088A110A12D0253008B1072F0897
:1006A000B40030088A110A126224AE30B400330854
:1006B000B5003208B6008A110A12F8253708A900D9
:1006C0002908AF008A110A125524AE30B40033084D
:1006D000B5003208B6008A110A12F8253708A900B9
:1006E0002908B0008A110A12552443308A110A12CF
:1006F00045272F088A110A12D0252F08B107300884
:100700008A110A12D0253008B1072F08B40030082A
:100710008A110A1262248A110A121D27AE30B4000F
:100720003308B5003208B6008A110A12F8253708D6
:10073000A9002908AF008A110A125524AE30B4006E
:100740003308B5003208B6008A110A12F8253708B6
:10075000A9002908B0008A110A12552444308A11D0
:100760000A1245272F088A110A12D0252F08B1072F
:1007700030088A110A12D0253008B1072F08B400BA
:1007800030088A110A126224AE30B4003308B50072
:100790003208B6008A110A12F8253708A90029087C
:1007A000AF008A110A125524AE30B4003308B500E8
:1007B0003208B6008A110A12F8253708A90029085C
:1007C000B0008A110A125524AE30B4003308B500C7
:1007D0003208B6008A110A12F8253708A90029083C
:1007E000FF3C8A110A12031DF72B1F30B30045305E
:1007F0008A110A1245272F088A110A12D0252F08BC
:10080000B10730088A110A12D0253008B1072F0825
:10081000B40030088A110A12622420308A110A12A8
:10082000452750308A110A1245274C308A110A1286
:10083000452741308A110A12452759308A110A1278
:1008400045273108F039AD002D088A110A12D0254C
:1008500031080F39AD002D088A110A12D0258A11EE
:100860000A12D22AA8168A110A12EA2701308A111E
:100870000A129227A8128A110A12EA278A110A126A
:1008800025278A110A12C12427138A110A12F62772
:100890008A110A1287184F2C8A110A12482C8A11C1
:1008A0000A127C288A110A12522C3208FF3C8A1143
:1008B0000A12031D602CB201B30A8A110A12612CBC
:1008C000B20A0800B5003408AC002C0E0F39AC0099
:1008D0003030AC072C088A110A12452734080F392A
:1008E000AC003030AC072C088A110A1245273508B5
:1008F000AC002C0E0F39AC003030AC072C088A113C
:100900000A12452735080F39AC003030AC072C08E7
:100910008A110A12452FB800B401B501B601103092
:10092000B90036088A110A12AD243A08B600350813
:100930008A110A12AD243A08B50034088A110A1245
:10094000AD243A08B400B80DB70DB60DB50DB40D11
:100950008A110A12B90B912C0800BA003A08033E1A
:10096000BB008A110A12BB1DB72C3B08BA003A081B
:10097000303EBB008A110A12BB1FC02C3B08BA00D4
:1009800008008A110A12252720308A110A124527E9
:1009900020308A110A12452720308A110A12452771
:1009A00054308A110A12452765308A110A124527E8
:1009B0006C308A110A12452765308A110A124527C0
:1009C0006D308A110A12452765308A110A124527AF
:1009D00074308A110A12452772308A110A1245278B
:1009E00069308A110A12452763308A110A12452795
:1009F0008A110A121D2720308A110A124527203039
:100A00008A110A12452753308A110A124527793074
:100A10008A110A12452773308A110A124527743049
:100A20008A110A12452765308A110A1245276D304E
:100A30008A110A12452720308A110A12452772307E
:100A40008A110A12452765308A110A12452761303A
:100A50008A110A12452764308A110A124527793013
:100A60008A110A12452754308A110A12D02565309E
:100A70008A110A12D0256C308A110A12D0256530ED
:100A80008A110A12D0256D308A110A12D0256530DC
:100A90008A110A12D02574308A110A12D0257230B8
:100AA0008A110A12D02569308A110A12D0256330C2
:100AB0008A110A12D02520308A110A12D02553300B
:100AC0008A110A12D02579308A110A12D025733082
:100AD0008A110A12D02574308A110A12D025653085
:100AE0008A110A12D0256D308A110A12D0252030C1
:100AF0008A110A12D02572308A110A12D025653067
:100B00008A110A12D02561308A110A12D025643068
:100B10008A110A12D02579308A110A12D02DB40018
:100B2000B4088A110A12031D972D4130B40034080D
:100B3000013C8A110A12031D9F2D4930B40034086C
:100B4000023C8A110A12031DA72D5130B40034084B
:100B5000033C8A110A12031DAF2D5930B40034082A
:100B6000043C8A110A12031DB72D6130B400340809
:100B70009F0001308A110A12A427831603138230C2
:100B80009F00831234089F001F151F19C52D1E08D2
:100B9000AA00831603131E088312AB0083120800F9
:100BA000B40034080C1ED22D8B138B1BD42D99004E
:100BB0008B1708000800B70034088A110A1217269C
:100BC00035088A110A124A268A110A125D26360849
:100BD0008A110A124A268A110A125D2637088A11DA
:100BE0000A124A268A110A125D268A110A12BD2E9D
:100BF000B70034088A110A12172635088A110A121A
:100C00004A268A110A125D2636088A110A124A26D5
:100C10008A110A125D2634088A110A1222268A11C4
:100C20000A122E263808B7008A110A12BD2EB80003
:100C30008A110A12E32638088A110A124A268A11F2
:100C40000A125D2EB8008A110A12E3263808013E06
:100C50008A110A124A268A110A125D2EB8008A11D8
:100C60000A127F2638108A110A12A01C382E381456
:100C70000830B9000310B80D8A110A127F26381007
:100C80008A110A12A01C452E38148A110A12B90BB7
:100C90003A2E0800B9000830BA00A0108A110A12D2
:100CA000B91F532EA0148A110A12A0260310B90DE1
:100CB0008A110A12BA0B4D2E08008A110A1209274E
:100CC00024168A150A1224208A110A120927A4154B
:100CD0008A150A1227208A110A1209278A110A1274
:100CE0008719752E8A110A126E2E8A110A12092787
:100CF000A4118A150A1227208A110A12092F8A11B3
:100D00000A12092724168A150A1224208A110A12A7
:100D10000927A0108A110A12071E8F2EA0148A110B
:100D20000A120927A4118A150A1227208A110A1209
:100D30000927A4158A150A1227208A110A12092FD9
:100D40008A110A12092724128A110A12A01CA92E3C
:100D500024168A150A1224208A110A120927A415BA
:100D60008A150A1227208A110A120927A4118A1546
:100D70000A1227208A110A12092F8A110A1209273A
:100D8000A4118A150A1227208A110A12092724128F
:100D90008A150A1224208A110A120927A4158A1515
:100DA0000A1227208A110A12092724168A150A1204
:100DB00024208A110A120927A4118A150A12272051
:100DC0008A110A12092F8A110A120927A4118A15F9
:100DD0000A1227208A110A12092724168A150A12D4
:100DE00024208A110A120927A4158A150A1227201D
:100DF0008A110A12092724128A150A1224208A113C
:100E00000A120927A4118A150A1227208A110A1228
:100E1000092F0C308A110A12DB2FA8118A110A122D
:100E2000F027A4118A150A12272028128A110A1203
:100E3000ED2724128A150A122428A8308A110A12D2
:100E4000532F80308A110A12532F08308A110A1248
:100E5000532701308A110A125327C8308A110A1207
:100E6000C72702308A110A125327C8308A110A1282
:100E7000C72706308A110A1253270C308A110A122A
:100E80005327C8308A110A12C72FB60027168A11B5
:100E90000A12FC27360E0F398A110A126927360802
:100EA0008A110A12692FB40027128A110A12FC272C
:100EB000340E0F398A110A12692782308A110A12F8
:100EC000C72734088A110A12692782308A110A1248
:100ED000C72FB700A7168A110A12F92737088A11F7
:100EE0000A12FF27A7128A110A12F927FA308A116B
:100EF0000A12DB2F00308A110A12FF2727128A11EB
:100F00000A12FC27A7128A110A12F92700308A1543
:100F10000A12102023128A150A123320A3128A15EE
:100F20000A123028B4003408B6006430B7000A3022
:100F30008A110A12AD2FB4003408B6006430B7002D
:100F400001308A110A12AD2FB5003508B6000A30FB
:100F5000B70001308A110A12AD2FB800FF30B90076
:100F60003708BB003608BA0017308A110A12390751
:100F70000318B72F8A110A12BA0BB42F8A110A125A
:100F8000BB0BB22F8A110A12B80BB02F0800B500A4
:100F90003508B600B6088A110A12031DD22F8A112D
:100FA0000A12DA2F0A308A110A12DB27B6038A11D5
:100FB0000A12CA2F0800BB00F430BC00FC30BD0090
:100FC0008A110A123B083C07031C00343D07031832
:100FD000E62F08008A150A120A288A150A120A281A
:100FE0008A150A120A288A150A120D288A150A1269
:100FF0000D288A150A120D288A150A120D28B80024
:1010000038080F39B9002708F0393904A7008A15C4
:101010000A120D2828088700080027088600080003
:10102000A90029080F39AA002308F0392A04A300CF
:101030008A150A123D288A150A123A288A150A12B8
:101040003A288A150A123A288A150A123A288A1565
:101050000A123A288A150A123D288A150A123D28D2
:101060008A150A123D288A150A123D28A2008A15FF
:101070000A124028240867000800230866000800B8
:101080002208650008008316031308008312031367
:02109000080056
:02400E00723FFF
:00000001FF
